:0300330002001AAE
:04001A0053D8EF3296
:100003008E118F12E5121512AE11700215114E608A
:0700130005120F8480EE22AC
:0300230002004692
:10004600C0E0C083C082C086758600C0D075D00867
:1000560030990E300B07A20E929B853699C299D223
:100066001220120302041EC21220030302024E20B3
:100076000B03020126E53AC39553503C200C34206D
:100086000931907F9BE055387029301012AF3A0540
:100096003A74402FF582E4347EF583E013920EAF76
:1000A6003A053A74402FF582E4347EF583E0F5365E
:1000B60002041CC20B02041C907FC7E4F0C203308A
:1000C6000D0CC20D907FBB04F0C20B02041C907F86
:1000D600C8E030E105C20B02041C907FC9E0F5536D
:1000E600907DC0E013920D7516FF200C2B20092879
:1000F600907F9BE055387020301011907DC1E01341
:03004300020E00AA
:03000000020026D5
:0C002600787FE4F6D8FD758154020B28A9
:40010600920EA3E0F536753A0302041C753A02907DC1E0F53602041C753A01C20B02041CE53AC3955350030201C9907FC6E030E107C214C20502041C907FC7E0F553907ECB
:4001460040E013920D7516FF200C7020096D907F9BE055387065301010907E41E013929BA3E0F599753A038009907E41E0F599753A02E53AC395534017907FC7E4F0C203F6
:40018600200D0302041CC20D907FBB04F002041C301012AF3A053A74402FF582E4347EF583E013920EAF3A053A74402FF582E4347EF583E0F536D20B02041C753A01C214A3
:4001C60002041C300C03020249200977907F9BE05538706F301012AF3A053A74402FF582E4347EF583E013929BAF3A053A74402FF582E4347EF583E0F599E53AC3955340AB
:4002060017907FC7E4F0C203200D0302041CC20D907FBB04F002041C301012AF3A053A74402FF582E4347EF583E013920EAF3A053A74402FF582E4347EF583E0F536D20B44
:4002460002041CC21402041C200B030202FFE53AC39553503C200C34200931907F9BE055387029301012AF3A053A74C02FF582E4347DF583E013920EAF3A053A74C02FF5F9
:4002860082E4347DF583E0F53602041CC20B02041C907FC9E4F0D203300D0CC20D907FBB04F0C20B02041C907FC6E030E105C20B02041C907FC7E0F553907E40E013920DAF
:4002C6007516FF200C2B200928907F9BE055387020301011907E41E013920EA3E0F536753A0302041C753A02907E41E0F53602041C753A01C20B02041CE53AC39553500381
:400306000203A2907FC8E030E107C214C20502041C907FC9E0F553907DC0E013920D7516FF200C7020096D907F9BE055387065301010907DC1E013929BA3E0F599753A037A
:400346008009907DC1E0F599753A02E53AC395534017907FC9E4F0D203200D0302041CC20D907FBB04F002041C301012AF3A053A74C02FF582E4347DF583E013920EAF3A81
:40038600053A74C02FF582E4347DF583E0F536D20B02041C753A01C21402041C200C75200972907F9BE05538706A301012AF3A053A74C02FF582E4347DF583E013929BAF02
:4003C6003A053A74C02FF582E4347DF583E0F599E53AC395534013907FC9E4F0D203300D35C20D907FBB04F0802C301012AF3A053A74C02FF582E4347DF583E013920EAF3D
:400406003A053A74C02FF582E4347DF583E0F536D20B8002C214D20120980302055AC2982002030204C7201627AF39053974802FF582E4347EF583E599F030104DAF3905C8
:400446003974802FF582E4347EF583E598F0803A859910E510B54704D209802EE510B54604C2098025AF39053974802FF582E4347EF583E510F0301011AF39053974802F11
:40048600F582E4347EF583E598F0D20FE539C395435003020558907FB8E030E116E539C39440500302055815391539052B433401020558907FB7E539F0753900C2020205D3
:4004C60058201627AF39053974002FF582E4347EF583E599F030104DAF39053974002FF582E4347EF583E598F0803A859910E510B54704D209802EE510B54604C209802573
:40050600AF39053974002FF582E4347EF583E510F0301011AF39053974002FF582E4347EF583E598F0D20FE539C395434024907FB6E030E112E539C3944040161539153909
:40054600052B433401800B907FB9E539F0753900D202D201300105C201020056D0D0D086D082D083D0E032907FBCE020E151E534604DE5317049E53430E108E4F52F7534D4
:4005860001800BA208E433F52FC208E4F534E4F5117E007B0074242511F9EE3400FA120D06FF74002511F582E4347DF583EFF00511E511B40CDB907FBD740CF075311090CD
:4005C6007FCAE030E1030206F3E4F51174402511F582E4347DF583E0FFE5117C007B00243BF9EC3400FAEF120D1F0511E511B418DBE53B601175C92075C836853CCA853D98
:40060600CBE4907F9FF0E53E139210929F853F38E540139216E5416009907F98E054FBF08007907F98E04404F0E5426009907F98E0547FF08007907F98E04480F0E54860BE
:400646000BC20CC209907F95E04402F0E549600CD209433401907F95E04402F0E54A600DC2AFC20BD200E4F553F53AD2AFE54B6005301602D209E54C6015907F95E054FDB4
:40068600F0907F9EE04402F0907F98E054FDF0E54D600AD29CC298752C0175311EE54E6007C29CE4F539F52CE54F6003E4F539E5506002D207E551600AE54D7002F531E55C
:4006C600514234E552601F907FD77411F07431F07412F07432F07413F07433F07414F07434F0D203D202D208E4907FCBF0A20CE433FF652960058F29433401A209E433FF84
:40070600652A60058F2A433401907F9BE0FF54086408FE652560058E25433401EF54106410FE652660058E26433401EF54406440FE652760058E27433401EF54206420FE1C
:40074600652860058E28433401907F9AE054406440FE652E60058E2E433401300735C2AF300218907FB8E020E127E5396009907FB7F0E4F539C202C2078016907FB6E0203B
:40078600E10FE5396009907FB9F0E4F539D202C207D2AF20053D30031E907FC6E020E133907E40E013920D753A01907FC7E0F553D2057516FF801C907FC8E020E115907DD3
:4007C600C0E013920D753A01907FC9E0F553D2057516FF201433200006E53A6553702A30051A300309E4907FC7F0C2038007E4907FC9F0D203C205E4F553F53A300D0AC265
:400806000DC200907FBB7401F0301403020914200503020914300C03020914300903020914907F9BE055386003020914300361301012AF3A053A74402FF582E4347EF5833F
:40084600E013921BAF3A053A74402FF582E4347EF583E0FEE53AC39553502A301012AF3A053A74402FF582E4347EF583E013920EAF3A053A74402FF582E4347EF583E0F546
:4008860036D20B806AC20BE4907FC7F0C203805F301012AF3A053A74C02FF582E4347DF583E013921BAF3A053A74C02FF582E4347DF583E0FEE53AC39553502A301012AFE7
:4008C6003A053A74C02FF582E4347DF583E013920EAF3A053A74C02FF582E4347DF583E0F536D20B8009C20BE4907FC9F0D203301004A21B929BD214C2AF8E99200B0D301D
:400906000D0AC20DC200907FBB7401F0D2AF22907FE9E0120D310A11000A7E010ADB030938060A020809F60909DE0A09ED0B00000B19907FEBE024FE601914605A24026041
:4009460003020B19740D907FD4F07487907FD5F0020B20907FEAE070047F0280027F037582D875830DEFF07582D175830DF07582CA75830DF07582C375830DF0907FEAE078
:400986000475829E75830DF0740D907FD4F07499907FD5F0020B20907FEAE0700B7511FF75120D7513DC801B907FEAE0B4010B7511FF75120D7513E080097511FF75120D19
:4009C6007513F0AA12A913AE02EE907FD4F0AF01EF907FD5F0020B20907F00E515F0907FB57401F0020B20907FEAE0F515020B20120CB1907FEAE0F514020B20907F00E5BF
:400A060014F0907FB57401F0020B20907FE8E0247F602714603424026003020B19A217E433FF25E0FFA219E4334F907F00F0E4A3F0907FB57402F0020B20E4907F00F0A3B7
:400A4600F0907FB57402F0020B20907FECE0F45480FFC4540FFFE054072F25E024B4F582E4347FF583E054FD907F00F0E4A3F0907FB57402F0020B20907FE8E024FE601726
:400A860024026003020B20907FEAE064016003020B19C217020B20907FEAE07076907FECE0F45480FFC4540FFFE054072F25E024B4F582E4347FF583E4F0907FECE05480D6
:400AC600FF131313541FFFE054072F907FD7F0E04420F08045907FE8E024FE601024027039907FEAE06401702AD217802D907FEAE07020907FECE0F45480FFC4540FFFE056
:400B060054072F25E024B4F582E4347FF5837401F08007907FB4E04401F0907FB4E04402F022C210E4F514F534C209C20CC20BC214C20DC216C211C207C212C20FC208F538
:400B460035F539F553F53AF533F530F52FF52EF52DF52CF52BF52AF529F528F527F526F525F524C205C218C21AC217C219C215C204D213C206C201907F92E054FDF0D2E820
:400B860043D820907FDE7401F0907FDFF0907FAB74FFF0907FA9F0907FAAF05391EF907FAFE04401F0907FAEE0440FF0907FAC740EF0D2AFD2BCD21B120F5FC21830040316
:400BC60012056D30042A300627C206E51660161516907FD8E030E6047F0080027F20907F96EFF08006907F967420F0120C0B80CD301807C21812091580C3301AC0C21A128E
:400C06000FBB80B922E53160021531E53960556535704BE533F460020533E533C395444043C2AF30021B907FB8E020E12D907FB7E539F0C202E4F539F533F5357516FF802D
:400C460019907FB6E020E112907FB9E539F0D202E4F539F533F5357516FFD2AF8006853935E4F533E52C6030200F07907F9BE030E00FE52D6006E4F52D433401E4F5308000
:400C860014E530D39545500DE530B54506752D014334010530C20F22907FD9E030E2047F0080027F20907F96EFF022E4907F93F0907F9C7430F0907F967420F0907F94748A
:400CC60001F0907F9D74BFF0907F977486F0907F957403F0907F9E7484F0907F98F0E4907FC7F0907FC9F0907FCBF075984043A810907FDE741FF0907FDF740FF0D204221A
:400D0600BB010689828A83E0225002E722BBFE02E32289828A83E49322BB010689828A83F0225002F722BBFE01F322D083D082F8E4937012740193700DA3A393F8740193EB
:400D4600F5828883E4737402936860EFA3A3A380DFC0E0C083C082C085C084C086758600907FC4E4F05391EF907FAB7404F0D086D084D085D082D083D0E03200000000007B
:400D86000012011001FF000040CD060C010100010200020902430001010080320904000007FF00000007050102400000070502024000000705030240000007058102400010
:400DC600010705820240000107058302400001070584024000010403090410034B00650079007300700061006E000E03530065007200690061006C000000020EA200020E41
:400E06007B00020D5700020EC900020E1000020E1400020E1800020E1C00020EF000020E2400020F1500020E2C00020F3AE4907F95F0907F94F0907F93F0907F9DE044020A
:400E4600F0907F97E04402F0907F9C7410F0E4907F96F0907F9D74FEF03017047F8080027F00907F97EFF0E4907F95F0907F9EF0907F98F022C0E0C083C082C085C084C00E
:400E8600867586005391EF907FAB7402F0D206D086D084D085D082D083D0E032C0E0C083C082C085C084C086758600D2185391EF907FAB7401F0D086D084D085D082D083EB
:400EC600D0E032C0E0C083C082C085C084C086758600D21A5391EF907FAB7408F0D086D084D085D082D083D0E032C0E0C083C082C085C084C0867586005391EF907FA974C2
:400F060002F0D086D084D085D082D083D0E032C0E0C083C082C085C084C0867586005391EF907FA97404F0D086D084D085D082D083D0E032C0E0C083C082C085C084C086D7
:400F46007586005391EF907FA97408F0D086D084D085D082D083D0E032907FD6E054FBF0E04408F0301B04E04402F07FF47E01120003907FD6E054F7F0E04404F0227400B9
:400F8600F58690FDA57C05A3E582458370F922907FD6E04480F0438701000000000022907FD6E04401F07F0D7E00120003907FD6E054FEF022120E33120F95907FD6E030FA
:090FC600E703120FA5120CB12281
:00000001FF
